:042CDE00C101C10768
:032D0400C2B42234
:032D0700D2B42221
:0D2C2100A2B4E43370047F0180027F002222
:1029D00075A40D7580FF75D44075A50C75F20F7543
:1029E000D50175F3F075A63075B0FF75E10675E297
:0229F000C22201
:102C030075BC4475E8C075BA1F75D10843E6082240
:0C2C620075A14075F80975A202D2AE22DF
:092CBD00E4F5B1F5A975B283221A
:0A2CB30075DA2175DB2143E61022DB
:0D2C2E007592077593F875910443E68022B6
:0B2C920075CA3475CBFFD2CAD2AD2248
:102AB000E4F5D9122CBD1229D0122C03122C62126B
:0B2AC0002CB31229AB122C92022C2E1A
:102BA400E4FEEF139293C292D292EFC313FF0EEEA0
:032BB400B408EF73
:012BB70022FB
:10271600752CFFE55C14600F14601114601324031C
:10272600700F532C7F800A532CBF8005532CDF80FB
:1027360000E55D14600F1460111460132403700F1C
:10274600532CEF800A532CF78005532CFB8000E5B1
:0B2756005B6003532CFCAF2C022BA493
:0D2C3B00754200754301854B2E854C2F22FC
:0D2C4800754400754501854D30854E3122E3
:0C2C6E00E4F542F543853A2E853B2F2209
:0C2C7A00E4F544F545853C30853D3122F1
:102B6400E55B6005E4F528F5297526007527011253
:062B74002C3B752B012231
:0D2C5500752800752901122C48752B0222EC
:102BCC00C202C204E4F547F548F526F527F52E7543
:032BDC002F0122A4
:102BDF00C203C206E4F549F54AF528F529F5307523
:032BEF003101228F
:061A1B00122BCC022BDFB0
:102B4C0075BB1175E8D030EDFDC2EDE5BED394C078
:082B5C004003D20922C2092244
:102B1A00121A1BE55B6003022B64E55C7003122B3F
:092B2A0064E55D7003122C5522D4
:082CC60090025DEFF0022CF218
:0E2C130090025DEFF01229F2122B1A02271622
:1025DD00E4FEFDAF050DEDB405F9AD070DEDC394AA
:1025ED000540F7E4FDAF050DEDB405F9AD070DEDB3
:1025FD00C3940540F775BB12E4FD75E8D030EDFDD1
:10260D00742D2DF582E43402F583E5BEF00D05BB86
:10261D00EDC3940240E490022DE0FDD394194021C6
:10262D00A3E0FCD394194019ED94CC5004C20A8058
:10263D0002D20AECC394CC5004C20B8008D20B809A
:10264D0004C20BC20AA20AE43325E0FEA20BE43356
:02265D004EFF2E
:01265F002258
:10276100EF25E0FFA209E4334FFFB4080050379092
:102771002777F828287302278F02279202279502CC
:10278100279802279B02279E0227A10227A47F38B0
:10279100227F39227F3A227F3B227F3C227F3D22CA
:0927A1007F3E227F3F227F382297
:1012A100122AB01225DD90022AEFF075460F753A29
:1012B10000753B01754B00754C01753C00753D0196
:1012C100754D00754E01121A1BC2A4C2A5750807FF
:1012D1007509D0122B4CE0FF12276190024FEFF0FD
:1012E100300903122D07D2AF43E601122B33122925
:1012F100F2122B1A122716300708122CF2122D07A0
:10130100C207E525606C14604D24FD603424FC6047
:101311001E24067057635B01121A1BE55B7004E51E
:101321005C7003122B64E55D7027122C5580220539
:101331005CE55CB40403E4F55C122BCC122B6480F5
:1013410010055DE55DB40403E4F55D122BDF122C9D
:1013510055122BB88016300113300910122C21EFD1
:101361006005122D078005122D04C21A122716E4FA
:08137100F5252000030214DA47
:10137900C200E50945086008E50915097002150864
:101389007D04E4FF120EAA7D057F01120EAA7D06D7
:101399007F02120EAA7D077F03120EAAE55E2513AE
:1013A900FEE43390022BF0A3CEF0C2AD90022BE005
:1013B900FEA3E0FF9008A875F00312192DEE75F051
:1013C90003A42583F583E493F53E740193F53F90D7
:1013D90008A775F003EF12192DEE75F003A4258304
:1013E900F583E493754B00F54CD2ADE5602512FE0B
:1013F900E43390022BF0A3CEF0C2AD90022BE0FEB5
:10140900A3E0FF9008A875F00312192DEE75F003FB
:10141900A42583F583E493F532740193F533900899
:10142900A775F003EF12192DEE75F003A42583F5C6
:1014390083E493753A00F53BD2ADE55F2514FEE4EC
:101449003390022BF0A3CEF0C2AD90022BE0FEA3A5
:10145900E0FF9008A875F00312192DEE75F003A4AA
:101469002583F583E493F540740193F5419008A72A
:1014790075F003EF12192DEE75F003A42583F5839A
:10148900E493754D00F54ED2ADE5612515FFE433C2
:10149900FE90022BF0A3EFF0C2AD9008A875F003FF
:1014A90012192DEE75F003A42583F583E493F53421
:1014B900740193F5359008A775F003EF12192DEE15
:1014C90075F003A42583F583E493753C00F53DD2BB
:0114D900AD65
:1014DA001228AFEF70030212F8900252E0FFB40B29
:1014EA0002D201EF6431703A90024FE0FF9002534A
:1014FA00E06F702E122ACB50FB90024FE0FF122BA6
:10150A008F900254E0FFA3E0FDA3E0FBA3E090026A
:10151A0030F0121BE1122ACB50FB90024FE0FF126F
:10152A002B7A900252E06432703490024FE0FF90BE
:10153A000253E06F7028122ACB50FB90024FE0FF53
:10154A00122B8F900254E0FFA3E0FDA3E0FB121FD1
:10155A002D122ACB50FB90024FE0FF122B7A9002F9
:10156A0052E0642D703990024FE0FF900253E06F11
:10157A00702D122ACB50FB90024FE0FF122B8F12D4
:10158A002ACB50FB900254E0FFA3E0FDA3E0FB123C
:10159A002278122ACB50FB90024FE0FF122B7A904E
:1015AA000252E0642E703990024FE0FF900253E03D
:1015BA006F702D122ACB50FB90024FE0FF122B8F37
:1015CA00122ACB50FB900254E0FFA3E0FDA3E0FBFC
:1015DA00122347122ACB50FB90024FE0FF122B7ABC
:1015EA00900252E030E71290022AE0700C20B4090F
:1015FA007B017A02795112219020B41C900252E0A8
:10160A0014600D047012900253E0FF122C1380082C
:10161A00900253E0FF122CC6900252E0B4140A3032
:10162A000905122D04C21AD201900252E064156013
:10163A00030212F82009030212F8122D070212F807
:10240C00E5B0540FF5246546600CE5246546F52AC5
:10241C00752D03852446E52D6052152DE52D704C48
:10242C00E52A30E11DE52420E11890024D30010928
:10243C007405F0A374DCF080077401F0A37477F0DA
:10244C00D205E52A30E308E52420E303752508E5E9
:10245C002A30E208E52420E20375250430090DE555
:10246C002A30E008E52420E003752501300536907C
:10247C00024EE024FFF090024DE034FFF0E5B05442
:10248C00026005752502C20590024DE07002A3E0C2
:10249C007013C20530010C90024FE0FF7D05122A2B
:1024AC00558002D207E53945386011E53915397088
:0C24BC000215381445387004D2A6D2A7CF
:0124C80022F1
:032D0A00D2FA22D8
:1019F300E549C4F854F0C8E54AC4540F48F5A39028
:0E1A0300024A74FFF0A3742DF0A3740AF022BF
:102AE600C2FAE549C4540F44A0F5A390024A74FF04
:0A2AF600F0A37419F0A374F3F022AA
:032D0D00D2FA22D5
:102A7500E547C4F854F0C8E548C4540F48F5A39099
:0E2A8500024A74FFF0A3742DF0A3740DF0222A
:102B0000C2FAE547C4540F4490F5A390024A74FFFB
:0A2B1000F0A3742AF0A37475F022FC
:031A15000227AAFB
:1027AA00C0E0C0F0C083C082C0D075D000C000C0F5
:1027BA0001C002C003C004C005C006C007C2FF9022
:1027CA00024AA3E0FAA3E0F912195FD007D006D0B3
:1027DA0005D004D003D002D001D000D0D0D082D00E
:0627EA0083D0F0D0E032C4
:061A2700D2A47536022274
:062CEC00D2A5753702229B
:031A1200021D9121
:101D9100C0E0C0F0C083C082C0D075D000C000C018
:101DA10001C002C003C004C005C006C007C2CF20E5
:101DB1000803021E69C208E5366005D53602C2A4D1
:101DC100E52745267003021E58E52F152F700215D1
:101DD1002E14452E6003021E58E5436401454270EE
:101DE1003D854B2E854C2FE55CB4020620860330E1
:101DF1000206122660EF605FE55B6008E52BB40127
:101E010003122C55E55B6006E52B64037049E55C24
:101E1100B4020620864120023E122C6E8039122C1B
:101E21006E12267AEF6030E55B600AE52BB4030F92
:101E3100752B048007300404C2048003121A27E5BD
:101E41005B6005E52BB4010FE55C7005122B648026
:101E51000675260075270090024A74FFF0A3742BC3
:101E6100F0A37400F0021F10D208E5376005D537E2
:101E710002C2A5E52945287003021F02E53115318B
:101E8100700215301445307078E5456401454470A1
:101E910041854D30854E31E55B700BE55DB4020641
:101EA100209003300306122695EF6055E55B60082C
:101EB100E52BB40203752B03E55B6006E52B640497
:101EC100703FE55DB40206209037200334122C7A6E
:101ED100802F122C7A1226AFEF6026122C48300682
:101EE10004C2068003122CECE55B6007E55C70031D
:101EF100122B64E55B7004E55D60067528007529A9
:101F01000090024A74FFF0A3742AF0A374E6F0D2A1
:101F1100FFD007D006D005D004D003D002D001D025
:0C1F210000D0D0D082D083D0F0D0E032CD
:031A2D0002283656
:10283600C0E0C0F0C083C082C0D075D000C000C068
:1028460001C002C003C004C005C006C00753917F83
:1028560012240C75BB0475E8D0D007D006D005D07D
:1028660004D003D002D001D000D0D0D082D083D003
:04287600F0D0E0328C
:031A21000228DFB9
:1028DF00C0E0C0D075D000C000C007C2EDAFBB7460
:1028EF000E2FF8A6BEE5BB640B600705BB75E8D0DD
:0D28FF008002D200D007D000D0D0D0E0324F
:031A24000229860E
:10298600C0E030D80BC2D8E55C64036003122B6448
:1029960030D90FC2D9E55B7009E55D6403600312A7
:0529A6002C55D0E032C9
:10266000E548253FF548E547353EF54740037F00FF
:10267000227F0174FFF547F54822C3E5489533F5FD
:1026800048E5479532F54740037F00227F017400FB
:10269000F547F54822E54A2541F54AE5493540F533
:1026A0004940037F00227F0174FFF549F54A22C3A8
:1026B000E54A9535F54AE5499534F54940037F00EB
:0A26C000227F017400F549F54A225B
:1008A7000133330131B601303A012EBD012D41012B
:1008B7002BC4012A480128CB01274F0125D2012447
:1008C700560122D901215D011FE0011E64011CE7C9
:1008D700011B6B0119EE0118720116F5011578015C
:1008E70013FC01127F011103010F86010E0A010C8F
:1008F7008D010B1101099401081801069B01051FC1
:100907000103A201050A0104F40104DF0104CA017D
:1009170004B50104A001048B0104760104600104FD
:100927004B01043601042101040C0103F70103E222
:100937000103CC0103B70103A201038D0103780171
:10094700036301034E01033801032301030E010270
:10095700F90102E40102CF0102BA0102A401028FE8
:1009670001027A01028801028101027A0102730100
:10097700026C01026501025E010257010250010289
:100987004901024201023B01023401022D01022604
:1009970001021F01021801021101020901020201ED
:1009A70001FB0101F40101ED0101E60101DF010194
:1009B700D80101D10101CA0101C30101BC0101B57F
:1009C7000101AE0101AB0101A101019701018D01F7
:1009D700018401017A01017001016601015C0101D5
:1009E7005201014801013F01013501012B0101219C
:1009F70001011701010D0101030100F90100F001D7
:100A070000E60100DC0100D20100C80100BE0100C0
:100A1700B40100AB0100A101009701008D01008323
:100A270001007901008001007D01007B0100780150
:100A3700007501007201006F01006D01006A01007D
:100A47006701006401006101005E01005C0100595B
:100A570001005601005301005001004E01004B01F7
:100A6700004801004501004201003F01003D01002F
:100A77003A01003701003401003101002F01002C39
:100A870001002901002B01002A010029010028018A
:100A97000027010026010025010024010023010091
:100AA7002201002102004002003E02003C02003AFF
:100AB700020038020036020034020032020030021F
:100AC700002E02002C03003F03003C030039030003
:100AD7003603003303003004003C040038040034BC
:100AE70005003D04003305003F05003D05003C05BA
:100AF700003A05003905003805003606003F0600B4
:100B07003E06003C06003A06003906003707003E5D
:100B170007003C07003A07003808003E08003C0879
:100B2700003A09003E09003C0A003F0A003D0B005D
:100B3700400B003C0C003F0C003B0D003C0E003D01
:100B47000F003D0E003C0F003F0F003D100040100E
:100B5700003E10003C11003F11003D12003F120003
:100B67003D13003E14004014003E15003F160040A0
:100B770016003D17003E18003E19003E1A003E1BA6
:100B8700003E1D00401E003F1F003E21003F230086
:100B97003F25003F27003F2A003F2D003F30003F01
:100BA70034003F30003F31004031004031004031D8
:100BB700004031003F31003F31003F31003F3100FD
:100BC7003F31003F320040320040320040320040A7
:100BD70032003F32003F32003F32003F32003F32A7
:100BE700003F3300403300403300403300403300C0
:100BF7003F33003F33003F33003F33003F33003F75
:100C070034004034004034004034003F34003F3467
:100C1700003F34003F34003F34003F35004035008B
:100C27004035004035003F35003F35003F35003F38
:100C370035003F360040360040360040360040362B
:100C4700003F36003F36003F36003F36003F370053
:100C57004037004037004037003F37003F37003FFD
:100C670037003F37003F38004038004038004038F1
:100C7700003F38003F38003F38003F38003F390019
:100C87004039004039004039003F39003F39003FC3
:100C970039003F3A00403A00403A00403A003F3AB4
:100CA700003F3A003F3A003F3B00403B00403B00DB
:100CB700403B00403B003F3B003F3B003F3C004088
:100CC7003C00403C00403C00403C003F3C003F3C77
:100CD700003F3D00403D00403D00403D003F3D009E
:100CE7003F3D003F3D003F3E00403E00403E00404C
:100CF7003E003F3E003F3E003F3F00403F00403F39
:100D070000403F003F3F003F3F003F400040400062
:100D17004040004040003F40003F40003F4100400E
:100D270041004041004041003F41003F41003F42F8
:100D3700004042004042004042003F42003F420024
:100D47003F43004043004043004043003F43003FD0
:100D570044004044004044004044003F44003F44B6
:100D6700003F45004045004045003F45003F4500E6
:100D77003F46004046004046004046003F46003F91
:100D870047004047004047003F47003F47003F4874
:100D9700004048004048003F48003F4900404900A4
:100DA7004049004049003F49003F4A00404A00404F
:100DB7004A00404A003F4B00404B00404B00404B2D
:100DC700003F4B003F4C00404C00404C003F4C0064
:100DD7003F4D00404D00404D00404D003F4E00400C
:100DE7004E00404E00404E003F4F00404F00404FE6
:100DF70000404F003F50004050004050004050001E
:100E07003F51004051004051003F51003F520040C8
:100E170052004052003F530040530040530040539C
:100E2700003F54004054004054003F54003F5500D9
:100E37004055004055003F56004056004056003F81
:100E470057004057004057003F57003F5800405851
:100E5700004058003F59004059004059003F5A0090
:100E6700405A00405A003F5B00405B00405B003F38
:100E77005C00405C00405C003F5D00405D00405D01
:100E8700003F5E00405E00405F00405F00405F0043
:100E97003F60004060004060003F610040610040EB
:030EA700620040A6
:1025560090022D7403F0E4A3F0FFA3F0122CCE7EBC
:102566003A7F007B017A02792D900235E4F0A304CC
:10257600F01227F0E4FF745E2FF8E4F60FEFB404D0
:10258600F5E4F55BF55CF55D90022EF090022EE029
:10259600FFC3941E5029EF75F007A42401F582E4C9
:1025A600343AAF82FE7B007A00795B900235E4F024
:1025B600A37407F01227F090022EE004F080CD7E7F
:1025C6003A7FD37B017A02792F900235E4F0A30497
:0725D600F01227F00229605A
:102BB800201A1030010820B408122CD68003122DD8
:042BC80004D21A22F7
:102B3300903AD3E493600C903A00E4936403600307
:092B4300122556E490025DF02217
:1029F20090025DE075F007A42401F9743A35F0FA0B
:102A02007BFF785B7C007D007E007F0712171AC275
:022A12001A2286
:10290C00122CCE90025DE075F007A42401F582E450
:10291C00343AAF82FE7B007A00795B900235E4F0AA
:0A292C00A37407F01227F0022960DF
:062CF20012290CC21A2297
:0A1BE10090022EEDF090022DEFF0BF
:101BEB00D39B5003021CBFE024FFFEE434FF9002A2
:101BFB0032F0A3CEF0EB14900231F090022EE024E1
:101C0B00FFFFE434FFFE900232E0FCA3E0FDD39F24
:101C1B00EE6480F8EC6480984003021D90903A01CA
:101C2B0075F007ED12192DEC75F007A42583AF8223
:101C3B00900239F0A3EFF0900231E075F007A42485
:101C4B0001F9743A35F0FA90023674FFF0A3EAF01A
:101C5B00A3E9F0E4900234F0A3F0900236A3E4750C
:101C6B00F001121786FEAFF0900239E475F0011205
:101C7B00178685F082F583E493FD12196590023582
:101C8B00E004F07006900234E004F0C3900235E0FB
:101C9B009407900234E0940040C012296090023304
:101CAB00E004F07006900232E004F0900231E004A0
:101CBB00F0021C0690022EE024FFFEE434FF90029B
:101CCB0032F0A3CEF0900230E014A3F090022DE09E
:101CDB0024FFFFE434FFFE900232E0FCA3E0FDC3DF
:101CEB009FEE6480F8EC6480985003021D90903A4C
:101CFB000175F007ED12192DEC75F007A42583AFD4
:101D0B0082900239F0A3EFF0900231E075F007A456
:101D1B002401F9743A35F0FA90023674FFF0A3EA15
:101D2B00F0A3E9F0E4900234F0A3F0900236A3E4C0
:101D3B0075F001121786FEAFF0900239E475F001D1
:101D4B0012178685F082F583E493FD1219659002D4
:101D5B0035E004F07006900234E004F0C3900235D5
:101D6B00E09407900234E0940040C0122960900286
:101D7B0033E024FFF0900232E034FFF0900231E0C8
:051D8B0014F0021CD75A
:011D90002230
:051F2D0090022DEDF013
:101F3200EF1490023AF0EB14A3F090022DE014FF9C
:101F420090023AE0D39F400302208AA3E075F00793
:101F5200A42401F582E4343AAF82FEE490023CF01C
:101F6200A3F090023CE0FCA3E0FDC39407EC9400D4
:101F7200502B0FEFAA0670010E14F5828A83E493A8
:101F8200FB74332DF582E43402F583EBF090023DCD
:101F9200E004F070CD90023CE004F080C590023B7A
:101FA200E075F007A42401F9743A35F0FA90022E94
:101FB20074FFF0A3EAF0A3E9F090023AE075F007AB
:101FC200A42401F582E4343AAF82900231F0A3EF07
:101FD200F0E490023CF0A3F090022EA3E475F0012D
:101FE200121786FEAFF0900231E475F001121786E7
:101FF20085F082F583E493FD12196590023DE004B9
:10200200F0700690023CE004F0C390023DE09407B9
:1020120090023CE0940040C090023AE075F007A4C0
:102022002401F9743A35F0FA90022E74FFF0A3EA13
:10203200F0A3E9F0E490023CF0A3F090023CE0FC53
:10204200A3E0FDC39407EC9400502D90022EA3E46C
:1020520075F001121786FEAFF074332DF582E43469
:1020620002F583E0FD12196590023DE004F070CBA9
:1020720090023CE004F080C312296090023AE0042E
:08208200F0A3E004F0021F3C92
:01208A002233
:0723470090022DEBF0AC0742
:10234E00A3E5C1F0A2AFE433A3F0AF05A3E4F0A37D
:10235E00EFF0E07F00FE900230F0A3EFF0AD04ED61
:10236E00FF900230EEF0A3EFF0C2AF43C15D9002DA
:10237E005D740FF0122CCE90025DE075F007A42470
:10238E0001F9743A35F0FA90023274FFF0A3EAF0D4
:10239E00A3E9F0E4A3F0900230E0FCA3E0FFECFD33
:1023AE0090022DE0FBE490023AF0D20A12208B90BC
:1023BE000236EFF0FD900232A3E475F0011217869B
:1023CE00FEAFF0121965900231E004F07006900233
:1023DE0030E004F0900235E004F0E0C3940740B61C
:1023EE0012296090025DE004F0E0C3941E408590D7
:0E23FE00022EE0F5C1A3E024FF92AF022CE511
:0722780090022DEBF0AC0712
:10227F00A3E5C1F0A2AFE433A3F0AF05900232E4BF
:10228F00F0A3EFF0E07F00FE900232F0A3EFF0AD8D
:10229F0004EDFF900232EEF0A3EFF0C2AF43C15D49
:1022AF0090025D740FF090025DE0FFC3941E5079B1
:1022BF00EF75F007A42401F582E4343AAF8290025F
:1022CF0034F0A3EFF0E4900230F0A3F0900232E08C
:1022DF00FCA3E0FFECFD90022DE0FB900234E475CF
:1022EF00F00112178685F082F583E49390023AF09D
:1022FF00C20A12208B900233E004F0700690023273
:10230F00E004F0900231E004F07006900230E00437
:10231F00F0C3900231E09407900230E0940040AC9B
:10232F0090025DE004F00222B590022EE0F5C1A309
:08233F00E024FF92AF022CE53F
:102A3500A2AFE433FDC2AF758F0375B7A575B7F1C6
:0F2A45008F828E83E4F0F58FAF05EF24FF92AF01
:012A5400225F
:102A1400A2AFE433FCC2AF758F0175B7A575B7F1EA
:102A24008F828E83EDF0E4F58FAF04EF24FF92AF35
:012A3400227F
:1026CA00900244EEF0A3EFF0A3ECF0A3EDF0EB4A96
:1026DA006039900244E0FEA3E0FFA3E0FCA3E0F52A
:1026EA00828C83E0FD122A14EB1B70011A900247B8
:1026FA00E004F07006900246E004F0900245E0041F
:0C270A00F070CB900244E004F080C32289
:082CCE00E4900000F0A3F022E5
:10296000900000E0FEA3E0FF122A35900000E0FE98
:10297000A3E0FF7C007D027B007A021226CAE4906D
:062980000000F0A3F022AC
:0A196500A90590023EEEF0A3EFF09A
:10196F00EE54FEFE900000E0FCA3E0FD7002EE6C72
:10197F006059ED4C600312296090023EE0FEEE5478
:10198F00FEFE7F00900000F0A3EFF0900240EEF01B
:10199F00A3EFF0A37400F0A37402F07F007E029017
:1019AF000240E475F00112178685F082F583E49307
:1019BF00FD900242E475F00112178685F082F583DF
:1019CF00EDF0EF1F70011EEF4E70D490023EE0FC61
:1019DF00A3E0FDEC5401FC74022DF58274003CF57C
:0319EF0083E9F099
:0119F20022D2
:1027F000900230EEF0A3EFF0A3EBF0A3EAF0A3E930
:10280000F090023574FFF5F012178645F0602690BF
:102810000230E475F001121786AFF0FE900232E04C
:10282000FBA3E475F001121786A9F0FA121740FD18
:0628300012196580CC22A4
:102A5500900248EFF0A3EDF07F0A1224C9900248D6
:102A6500E0FF1224C9900249E0FF1224C9022CE5B7
:082CD6007F021224C9022CE563
:0628AF00122CF8EF602777
:1028B50090022D7402F0A37451F012293690022D66
:1028C500E475F00112178685F082F583EFF0122C7E
:0728D500FEEF70E67F012217
:0328DC007F002258
:102B7A0090022DEFF07F2F1224C990022DE0FF1250
:052B8A0024C9022CE546
:102B8F0090022DEFF07F301224C990022DE0FF123A
:052B9F0024C9022CE531
:022CE200C11817
:102ACB00E552B55614E551B5550FE552B55A0AE521
:0B2ADB0051B5590520C502D322C322CB
:0C2C8600758920438E08758DE8D28E22DF
:102BF20075C101E4F5C2F5C053C17F43C180022C07
:012C0200864B
:1029AB007E027F028E538F548E578F588E4F8F50CF
:1029BB007E027F168E558F568E598F5A8E518F529F
:0529CB00C217022BF20F
:10287A000558E558AA577002055714F5828A83EF5E
:10288A00F0AF050558E558AC577002055714F582A4
:10289A008C83EFF07416B5580B7402B5570675574A
:0528AA00027558022236
:072CE500C217C2C4D2C522D0
:1024C900201745D217055AE55AAC59700205591417
:1024D900F5828C8374FFF07C027D2AEDB55A0AECF3
:1024E900B55906755902755A16055AE55AAA597009
:1024F90002055914F5828A83E4F0EDB55A0AECB560
:102509005906755902755A16055AE55AAC59700299
:10251900055914F5828C83E4F07C027D2AEDB55AC5
:102529000AECB55906755902755A16055AE55AAA9B
:10253900597002055914F5828A83EFF0EDB55A0AEC
:0D254900ECB55906755902755A167F01222E
:102A9300E550B55408E54FB553037F0022855482B2
:0D2AA300855383E0B507037F01227F0022E9
:102936000554E554700205530554E554AE53700230
:10294600055314F5828E83E0FF7416B5540B74029A
:09295600B55306755302755402D5
:01295F002255
:062CF8007FFF122A932267
:062CFE00E4FF122A9322FC
:031A1800021A307F
:101A3000C0E0C083C082C0D075D000C000C002C06A
:101A400004C005C006C007E5C054FE1219391BA822
:101A5000081BA80A1BBE0C1BBE0E1B87101B87127F
:101A60001B9A141B9A161B7F1C1B7F1E1B7B241B9F
:101A70007B261B3C281B3C2A1B4A2C1B4A2E1ACABD
:101A8000C01AD7C21A8EE01A8EE200001BCAC2C565
:101A90000552E552700205517E027F2AB5070AEE13
:101AA000B551067551027552160552E552AC51708A
:101AB00002055114F5828C83E0F5C2EF6552700384
:101AC000EE65516003021BCA8069855551855652E7
:101AD000D2C4D2C5021BCAE552B55A12E551B55956
:101AE0000D855955855A56C2C5D2C4021BCA8552A6
:101AF00082855183E0B4FF03021BC60552E5527094
:101B00000205517E027F2AB5070AEEB551067551CE
:101B1000027552160552E552AC517002055114F58A
:101B2000828C83E0F5C2EF65527003EE655160036D
:101B3000021BCA755102755216021BCAE5C2602A01
:101B400090024FE065C2602280168555518556523D
:101B5000C2C5D218E5C2601290024FE065C2600AA9
:101B6000C2C4C2C5C2C1C2198060ADC27FFF122803
:101B70007AC2C4C2C5D2C1D219804FD2C5804B85AA
:101B80005155855256804385574F855850C2C4C21F
:101B9000C1301836D2C5C21880308555518556528D
:101BA000C2C4C2C1D2C58022C2C4C2C5201904C2E7
:101BB000C18017ADC2E4FF12287AD2C1800C8555CE
:101BC00051855652C2C1C2C4D2C5C2C0D007D006C8
:101BD000D005D004D002D000D0D0D082D083D0E0C5
:011BE00032D2
:0B2C9D00C2A6D2A775380B7539B8220B
:0B2CA800D2A6C2A775380B7539B82200
:070EAA0090022DEFF0AB05F3
:100EB100C2AFC212E0FF240AF8E690025CF0FD74B2
:100EC100122BF8E6F9C39DFCE4940090022EF0A3E6
:100ED100CCF030134D90022EE0FCA3E0FDC3EC6496
:100EE100809480502E740E2FF8E6700276039002E3
:100EF1002DE0FF240EF816E66003020F86740E2F14
:100F0100F8760174122BF8E6FE740A2FF8A606D2C1
:100F1100128072D3ED9404EC64809480405EC2131D
:100F2100804D90022EE0FEA3E0FFD39400EE64809A
:100F31009480402E90022DE0240EF8E67002760394
:100F410090022DE0FD240EF816E67039740E2DF88E
:100F5100760174122BF8E6FC740A2DF8A604D2125D
:100F61008023C3EF94FCEE6480947F500FD21390E2
:100F7100022DE0240AF8A601D212800990022DE088
:100F8100240EF8E4F6E5094508600302129E2012DA
:100F91000302129E90022DE0FD245EF8E6FE7458D5
:100FA1002DF582E43402F583E0FDEDFFE4FCFD90D4
:100FB10002301218F090022EE0FEA3E0FFD394005D
:100FC100EE6480948050030210D2EE3395E0FDFC74
:100FD10078101218DD9002341218F0900234E0FCFF
:100FE100A3E0FDA3E0FEA3E0FFC006C00790025C02
:100FF100E0FFC374FF9FFFE49400AB07FAE4F9F844
:10100100D007D0061218279002341218F09002343B
:10101100E0F8A3E0F9A3E0FAA3E0FBC00090022D01
:10102100E0245EF8E6FFC374FF9FFFE49400FEE452
:10103100FCFDD00012179C9002341218F090022D82
:10104100E0245EF8E6FF90025CE0D39F900234E07A
:10105100FCA3E0FDA3E0FEA3E0FFE440067B407AB1
:101061000180037BC0FAF9F812179C900234121820
:10107100F0900230E0F8A3E0F9A3E0FAA3E0FBC0AE
:1010810000A3E0FCA3E0FDA3E0FEA3E0FF781012C3
:1010910018CAD000EB2FFFEA3EFEE93DFDE83CFC1B
:1010A1009002301218F0E47FFF7EFFFDFC900230C9
:1010B100E0F8A3E0F9A3E0FAA3E0FBD31218B950DA
:1010C100030211E09002301218FC0000FFFF021130
:1010D100E090022EE0FEA3E0FFC3E49FFFE49EFE4A
:1010E1003395E0FDFC78101218DD9002341218F0EF
:1010F100900234E0FCA3E0FDA3E0FEA3E0FFC00703
:1011010090025CE0FBE4FAF9F8D00712182790028C
:10111100341218F0900234E0F8A3E0F9A3E0FAA346
:10112100E0FBC00090022DE0245EF8E6FFE4FCFD48
:10113100FED00012179C9002341218F090022DE09C
:10114100245EF8E6FF90025CE0C39F900234E0FC6D
:10115100A3E0FDA3E0FEA3E0FFE450067B407A019B
:1011610080037BC0FAF9F812179C9002341218F030
:10117100900230E0FCA3E0FDA3E0FEA3E0FFC00489
:10118100C005C006C007A3E0FCA3E0FDA3E0FEA3E9
:10119100E0FF78101218CAA804A905AA06AB07D067
:1011A10007D006D005D004C3EF9BFFEE9AFEED9960
:1011B100FDEC98FC9002301218F0E47FFF7EFFFDF9
:1011C100FC900230E0F8A3E0F9A3E0FAA3E0FBD33E
:1011D1001218B9400A9002301218FC000000009069
:1011E1000230A3A3A3E0FF90022DE0FB2458F58277
:1011F100E43402F583EFF0900230E0FCA3E0FDA3BC
:10120100E0FEA3E0FF78081218CA9002301218F02D
:10121100745E2BF8E6FFE4FCFDFE900230E0F8A3DB
:10122100E0F9A3E0FAA3E0FBC31218B9601490023D
:1012310030A3A3A3E0FF90022DE0245EF8A60712DD
:101241002BB830132A90022DE0FF240AF8E6FE2481
:1012510004FDE433FC745E2FF8E6FFD39DEC64805B
:10126100F87480984002801BEFC39E502980229021
:10127100022DE0FF240AF8E6FE745E2FF8E6FFD3A4
:101281009E4005122C9D8015EE24FCFEEFC39E505E
:0F12910005122CA88007D2A6D2A7122716D2AF1B
:0112A000222B
:03000000020800F3
:03000300021A03DB
:03000B00021A06D0
:03001300021A09C5
:03001B00021A0CBA
:03002300021A0FAF
:03002B00021A12A4
:03003300021A1599
:03003B00021A188E
:03004300021A1B83
:03004B00021A1E78
:03005300021A216D
:03005B00021A2462
:03006300021A2757
:03006B00021A2A4C
:03007300021A2D41
:10080000E4F5D9E5EF7480F5FF7402F5EF787FE445
:10081000F6D8FD9000007F007E04E4F0A3DFFCDE4C
:07082000FA75816102086214
:0B21900090022DEBF0A3EAF0A3E9F0B1
:10219B00900001121759900232F0E0FF540FA3F098
:1021AB00900003121759900234F0EF54F0649070C2
:1021BB0055E06052900233E030E30D20090A122BF8
:1021CB0064121A27D202D204900233E030E20D20BF
:1021DB00090A122C55122CECD203D206900233E0D2
:1021EB0030E10D30090A122B64121A27D202D204E5
:1021FB00900233E030E073300970122C55122CEC46
:10220B00D203D2068064900232E054F0FF64806007
:10221B000BEF64907030900234E0702A900233E040
:10222B00FF30E305200902C202EF30E2052009026C
:10223B00C203EF30E105300902C202EF30E02B3070
:10224B000928C2038024900232E054F0FFBFB01A79
:10225B0090022DE0FBA3E0FAA3E0F9900003121724
:0C226B0059FF900230E4F0A3EFF07F0078
:012277002244
:08208B00900237EFF0A3EDF025
:10209300A20A920EC210201CFDD21C90023BEBF050
:1020A300C20BD20CD20F7F01C2C4C211D2C530C041
:1020B300FDE5C054F02480700302214524C0601B59
:1020C30024E0600302217590023BE0F5C2A20BE419
:1020D3003342C2C2C5E4A3F002217730C1593011A3
:1020E30007D2C5C211022177300C0CC20CD20D905D
:1020F3000238E0F5C2807D300D11C20D900237E049
:10210300F5C2300E6FD211D20B8069200B66EFFD42
:1021130090023CE0FB3395E0FAC3EB9D7480F86AD0
:1021230098500E90023AE0F5C290023CE004F08031
:1021330043D2C4C21C803D300F04D2C58036D210B6
:102143008032EFFD90023CE0FB3395E0FAC3EB9D58
:102153007480F86A98500CA3E5C2F090023CE00446
:10216300F0D2C190023CE0B5070AC21CC2C1D2C47E
:102173008002D21030100853C0BF43C040C21CC2FB
:0C218300C0301C030220B190023DE0FFC0
:01218F00222D
:100827000212A1E493A3F8E493A34003F68001F234
:1008370008DFF48029E493A3F85407240CC8C333D2
:10084700C4540F4420C8834004F456800146F6DFA1
:10085700E4800B0102040810204080902CDEE47E27
:10086700019360BCA3FF543F30E509541FFEE49396
:10087700A360010ECF54C025E060A840B8E493A35D
:10088700FAE493A3F8E493A3C8C582C8CAC583CA88
:10089700F0A3C8C582C8CAC583CADFE9DEE780BE40
:012CE40000EF
:10164A00E709F608DFFA8046E709F208DFFA803E82
:10165A0088828C83E709F0A3DFFA8032E309F6086F
:10166A00DFFA8078E309F208DFFA807088828C83D7
:10167A00E309F0A3DFFA806489828A83E0A3F6088B
:10168A00DFFA805889828A83E0A3F208DFFA804C65
:10169A0080D280FA80C680D4806980F2803380103C
:1016AA0080A680EA809A80A880DA80E280CA8033A5
:1016BA0089828A83ECFAE493A3C8C582C8CCC5831D
:1016CA00CCF0A3C8C582C8CCC583CCDFE9DEE780ED
:1016DA000D89828A83E493A3F608DFF9ECFAA9F06C
:1016EA00EDFB2289828A83ECFAE0A3C8C582C8CCC2
:1016FA00C583CCF0A3C8C582C8CCC583CCDFEADEDB
:10170A00E880DB89828A83E493A3F208DFF980CC3C
:10171A0088F0EF60010E4E60C388F0ED2402B40435
:10172A000050B9F582EB2402B4040050AF232345DC
:06173A00822390169A7351
:10174000BB010689828A83E0225002E722BBFE02A7
:09175000E32289828A83E49322DA
:10175900BB010CE58229F582E5833AF583E0225045
:1017690006E92582F8E622BBFE06E92582F8E2228F
:0D177900E58229F582E5833AF583E49322A9
:10178600A3F8E0C5F025F0F0E58215827002158316
:06179600E0C838F0E82273
:10179C00E88FF0A4CC8BF0A42CFCE98EF0A42CFCEC
:1017AC008AF0EDA42CFCEA8EF0A4CDA8F08BF0A46A
:1017BC002DCC3825F0FDE98FF0A42CCD35F0FCEBC9
:1017CC008EF0A4FEA9F0EB8FF0A4CFC5F02ECD398E
:0F17DC00FEE43CFCEAA42DCE35F0FDE43CFC22FB
:1017EB0075F008758200EF2FFFEE33FECD33CDCCB5
:1017FB0033CCC58233C5829BED9AEC99E582984038
:10180B000CF582EE9BFEED9AFDEC99FC0FD5F0D614
:10181B00E4CEFBE4CDFAE4CCF9A88222B800C1B93E
:10182B000059BA002DEC8BF084CFCECDFCE5F0CB7C
:10183B00F97818EF2FFFEE33FEED33FDEC33FCEBB5
:10184B0033FB10D703994004EB99FB0FD8E5E4F970
:10185B00FA227818EF2FFFEE33FEED33FDEC33FC5D
:10186B00C933C910D7059BE99A4007EC9BFCE99A51
:10187B00F90FD8E0E4C9FAE4CCFB2275F010EF2F96
:10188B00FFEE33FEED33FDCC33CCC833C810D70796
:10189B009BEC9AE899400AED9BFDEC9AFCE899F8D1
:0E18AB000FD5F0DAE4CDFBE4CCFAE4C8F92264
:1018B900EB9FF5F0EA9E42F0E99D42F0E89C45F085
:0118C90022FC
:1018CA00E8600FECC313FCED13FDEE13FEEF13FFFC
:0318DA00D8F12220
:1018DD00E8600FEFC333FFEE33FEED33FDEC33FC69
:0318ED00D8F1220D
:0C18F000ECF0A3EDF0A3EEF0A3EFF0226B
:1018FC00A8828583F0D083D0821219131219131287
:10190C001913121913E473E493A3C583C5F0C583AB
:10191C00C8C582C8F0A3C583C5F0C583C8C582C835
:01192C002298
:0C192D00A42582F582E5F03583F58322C5
:10193900D083D082F8E4937012740193700DA3A33D
:1019490093F8740193F5828883E473740293686051
:06195900EFA3A3A380DF51
:06195F008A838982E47313
:00000001FF
